 setlocal004

 Timestamp is e53beb5f (reproducible build file hash)

 Preferred load address is 0000000180000000

 Start         Length     Name                   Class
 0001:00000000 00002f10H .text$mn                CODE
 0001:00002f10 00000036H .text$mn$00             CODE
 0001:00002f46 00000092H .text$x                 CODE
 0002:00000000 00000198H .idata$5                DATA
 0002:00000198 00000038H .00cfg                  DATA
 0002:000001d0 00000008H .CRT$XCA                DATA
 0002:000001d8 00000008H .CRT$XCZ                DATA
 0002:000001e0 00000008H .CRT$XIA                DATA
 0002:000001e8 00000008H .CRT$XIC                DATA
 0002:000001f0 00000008H .CRT$XIZ                DATA
 0002:000001f8 00000008H .CRT$XLA                DATA
 0002:00000200 00000008H .CRT$XLZ                DATA
 0002:00000208 00000008H .CRT$XPA                DATA
 0002:00000210 00000008H .CRT$XPZ                DATA
 0002:00000218 00000008H .CRT$XTA                DATA
 0002:00000220 00000010H .CRT$XTZ                DATA
 0002:00000228 00000000H .gehcont$y              DATA
 0002:00000228 00000000H .gfids$y                DATA
 0002:00000230 00001cd0H .rdata                  DATA
 0002:00001f00 00000000H .rdata$CastGuardVftablesA DATA
 0002:00001f00 00000000H .rdata$CastGuardVftablesC DATA
 0002:00001f00 00000028H .rdata$T                DATA
 0002:00001f28 000000a4H .rdata$voltmd           DATA
 0002:00001fcc 0000031cH .rdata$zzzdbg           DATA
 0002:000022e8 00000008H .rtc$IAA                DATA
 0002:000022f0 00000008H .rtc$IZZ                DATA
 0002:000022f8 00000008H .rtc$TAA                DATA
 0002:00002300 00000008H .rtc$TZZ                DATA
 0002:00002308 00000004H .tls                    DATA
 0002:0000230c 00000004H .tls$                   DATA
 0002:00002310 00000008H .tls$ZZZ                DATA
 0002:00002318 000002f8H .xdata                  DATA
 0002:00002610 000003e0H .edata                  DATA
 0002:000029f0 00000064H .idata$2                DATA
 0002:00002a54 00000014H .idata$3                DATA
 0002:00002a68 00000198H .idata$4                DATA
 0002:00002c00 0000041eH .idata$6                DATA
 0003:00000000 00000080H .data                   DATA
 0003:00000080 0001b378H .bss                    DATA
 0004:00000000 00000390H .pdata                  DATA

  Address         Publics by Value              Rva+Base               Lib:Object

 0000:00000000       __AbsoluteZero             0000000000000000     <absolute>
 0000:00000000       ___safe_se_handler_count   0000000000000000     <absolute>
 0000:00000000       ___safe_se_handler_table   0000000000000000     <absolute>
 0000:00000000       __arm64x_extra_rfe_table   0000000000000000     <absolute>
 0000:00000000       __arm64x_extra_rfe_table_size 0000000000000000     <absolute>
 0000:00000000       __arm64x_native_entrypoint 0000000000000000     <absolute>
 0000:00000000       __arm64x_redirection_metadata 0000000000000000     <absolute>
 0000:00000000       __arm64x_redirection_metadata_count 0000000000000000     <absolute>
 0000:00000000       __dynamic_value_reloc_table 0000000000000000     <absolute>
 0000:00000000       __enclave_config           0000000000000000     <absolute>
 0000:00000000       __guard_check_icall_a64n_fptr 0000000000000000     <absolute>
 0000:00000000       __guard_eh_cont_count      0000000000000000     <absolute>
 0000:00000000       __guard_eh_cont_table      0000000000000000     <absolute>
 0000:00000000       __guard_fids_count         0000000000000000     <absolute>
 0000:00000000       __guard_fids_table         0000000000000000     <absolute>
 0000:00000000       __guard_iat_count          0000000000000000     <absolute>
 0000:00000000       __guard_iat_table          0000000000000000     <absolute>
 0000:00000000       __guard_longjmp_count      0000000000000000     <absolute>
 0000:00000000       __guard_longjmp_table      0000000000000000     <absolute>
 0000:00000000       __hybrid_auxiliary_iat     0000000000000000     <absolute>
 0000:00000000       __hybrid_auxiliary_iat_copy 0000000000000000     <absolute>
 0000:00000000       __hybrid_code_map          0000000000000000     <absolute>
 0000:00000000       __hybrid_code_map_count    0000000000000000     <absolute>
 0000:00000000       __x64_code_ranges_to_entry_points 0000000000000000     <absolute>
 0000:00000000       __x64_code_ranges_to_entry_points_count 0000000000000000     <absolute>
 0000:00000100       __guard_flags              0000000000000100     <absolute>
 0000:00000000       __ImageBase                0000000180000000     <linker-defined>
 0001:00000000       ?NewObject@JNIEnv_@@QEAAPEAV_jobject@@PEAV_jclass@@PEAU_jmethodID@@ZZ 0000000180001000 f i libsetlocal004.obj
 0001:00000028       ?SetEventNotificationMode@_jvmtiEnv@@QEAA?AW4jvmtiError@@W4jvmtiEventMode@@W4jvmtiEvent@@PEAV_jobject@@ZZ 0000000180001028 f i libsetlocal004.obj
 0001:00000034       ?TranslateError@@YAPEBDW4jvmtiError@@@Z 0000000180001034 f   libsetlocal004.obj
 0001:000002ec       ?nsk_jni_check_exception@@YAHPEAUJNIEnv_@@QEBDH@Z 00000001800012ec f   libsetlocal004.obj
 0001:00000430       ?nsk_jni_lverify@@YAHHPEAUJNIEnv_@@HQEBDH1ZZ 0000000180001430 f   libsetlocal004.obj
 0001:000004d0       Agent_Initialize           00000001800014d0 f   libsetlocal004.obj
 0001:0000065c       Agent_OnAttach             000000018000165c f   libsetlocal004.obj
 0001:0000065c       Agent_OnLoad               000000018000165c f   libsetlocal004.obj
 0001:00000664       Breakpoint                 0000000180001664 f   libsetlocal004.obj
 0001:00000960       Java_nsk_jvmti_SetLocalVariable_setlocal004_getReady 0000000180001960 f   libsetlocal004.obj
 0001:00000a3c       Java_nsk_jvmti_SetLocalVariable_setlocal004_getRes 0000000180001a3c f   libsetlocal004.obj
 0001:00000a44       Java_nsk_jvmti_unit_FollowReferences_FollowRefObjects_addRefToVerify 0000000180001a44 f   libsetlocal004.obj
 0001:00000c1c       Java_nsk_jvmti_unit_FollowReferences_FollowRefObjects_getTag 0000000180001c1c f   libsetlocal004.obj
 0001:00000cdc       Java_nsk_jvmti_unit_FollowReferences_FollowRefObjects_resetRefsToVerify 0000000180001cdc f   libsetlocal004.obj
 0001:00000ce4       Java_nsk_jvmti_unit_FollowReferences_FollowRefObjects_resetTags 0000000180001ce4 f   libsetlocal004.obj
 0001:00000d28       Java_nsk_jvmti_unit_FollowReferences_FollowRefObjects_setTag 0000000180001d28 f   libsetlocal004.obj
 0001:00000f80       Java_nsk_share_jvmti_ArgumentHandler_getAgentOptionsString 0000000180001f80 f   libsetlocal004.obj
 0001:00001030       Java_nsk_share_jvmti_DebugeeClass_checkStatus 0000000180002030 f   libsetlocal004.obj
 0001:000010b8       Java_nsk_share_jvmti_DebugeeClass_resetAgentData 00000001800020b8 f   libsetlocal004.obj
 0001:00001118       Java_nsk_share_jvmti_RedefineAgent_agentStatus 0000000180002118 f   libsetlocal004.obj
 0001:00001124       Java_nsk_share_jvmti_RedefineAgent_isRedefined 0000000180002124 f   libsetlocal004.obj
 0001:00001130       Java_nsk_share_jvmti_RedefineAgent_redefineAttempted 0000000180002130 f   libsetlocal004.obj
 0001:0000113c       MA_checkStatus             000000018000213c f   libsetlocal004.obj
 0001:000011e0       __local_stdio_printf_options 00000001800021e0 f i libsetlocal004.obj
 0001:0000141c       exitOnError                000000018000241c f   libsetlocal004.obj
 0001:000014d0       fprintf                    00000001800024d0 f i libsetlocal004.obj
 0001:00001514       nsk_jvmti_lverify          0000000180002514 f   libsetlocal004.obj
 0001:00001604       nsk_jvmti_resetAgentData   0000000180002604 f   libsetlocal004.obj
 0001:00001684       nsk_jvmti_setFailStatus    0000000180002684 f   libsetlocal004.obj
 0001:000016c0       nsk_lcomplain              00000001800026c0 f   libsetlocal004.obj
 0001:000016e0       nsk_ldisplay               00000001800026e0 f   libsetlocal004.obj
 0001:00001700       nsk_ltrace                 0000000180002700 f   libsetlocal004.obj
 0001:00001720       nsk_lvcomplain             0000000180002720 f   libsetlocal004.obj
 0001:000018d8       nsk_lvdisplay              00000001800028d8 f   libsetlocal004.obj
 0001:00001924       nsk_lverify                0000000180002924 f   libsetlocal004.obj
 0001:00001980       nsk_lvtrace                0000000180002980 f   libsetlocal004.obj
 0001:000019e0       nsk_printf                 00000001800029e0 f   libsetlocal004.obj
 0001:00001a08       nsk_vprintf                0000000180002a08 f   libsetlocal004.obj
 0001:00001abc       printf                     0000000180002abc f i libsetlocal004.obj
 0001:00001fe4       __raise_securityfailure    0000000180002fe4 f   MSVCRT:gs_report.obj
 0001:00002018       __report_gsfailure         0000000180003018 f   MSVCRT:gs_report.obj
 0001:00002258       __GSHandlerCheck           0000000180003258 f   MSVCRT:gshandler.obj
 0001:00002278       __GSHandlerCheckCommon     0000000180003278 f   MSVCRT:gshandler.obj
 0001:000022f0       __security_check_cookie    00000001800032f0 f   MSVCRT:amdsecgs.obj
 0001:00002630       _DllMainCRTStartup         0000000180003630 f   MSVCRT:dll_dllmain.obj
 0001:00002670       __scrt_acquire_startup_lock 0000000180003670 f   MSVCRT:utility.obj
 0001:000026ac       __scrt_dllmain_after_initialize_c 00000001800036ac f   MSVCRT:utility.obj
 0001:000026e0       __scrt_dllmain_before_initialize_c 00000001800036e0 f   MSVCRT:utility.obj
 0001:000026f8       __scrt_dllmain_crt_thread_attach 00000001800036f8 f   MSVCRT:utility.obj
 0001:00002720       __scrt_dllmain_crt_thread_detach 0000000180003720 f   MSVCRT:utility.obj
 0001:00002738       __scrt_dllmain_exception_filter 0000000180003738 f   MSVCRT:utility.obj
 0001:00002798       __scrt_dllmain_uninitialize_c 0000000180003798 f   MSVCRT:utility.obj
 0001:000027c8       __scrt_dllmain_uninitialize_critical 00000001800037c8 f   MSVCRT:utility.obj
 0001:000027dc       __scrt_initialize_crt      00000001800037dc f   MSVCRT:utility.obj
 0001:00002828       __scrt_initialize_onexit_tables 0000000180003828 f   MSVCRT:utility.obj
 0001:000028b4       __scrt_is_nonwritable_in_current_image 00000001800038b4 f   MSVCRT:utility.obj
 0001:0000294c       __scrt_release_startup_lock 000000018000394c f   MSVCRT:utility.obj
 0001:00002970       __scrt_uninitialize_crt    0000000180003970 f   MSVCRT:utility.obj
 0001:0000299c       _onexit                    000000018000399c f   MSVCRT:utility.obj
 0001:000029d8       atexit                     00000001800039d8 f   MSVCRT:utility.obj
 0001:000029f0       __crt_debugger_hook        00000001800039f0 f   MSVCRT:utility_desktop.obj
 0001:000029f8       __scrt_fastfail            00000001800039f8 f   MSVCRT:utility_desktop.obj
 0001:00002b44       _guard_check_icall_nop     0000000180003b44 f i MSVCRT:guard_support.obj
 0001:00002b48       __security_init_cookie     0000000180003b48 f   MSVCRT:gs_support.obj
 0001:00002bf4       DllMain                    0000000180003bf4 f   MSVCRT:dll_dllmain_stub.obj
 0001:00002c18       ?__scrt_initialize_type_info@@YAXXZ 0000000180003c18 f   MSVCRT:tncleanup.obj
 0001:00002c28       ?__scrt_uninitialize_type_info@@YAXXZ 0000000180003c28 f   MSVCRT:tncleanup.obj
 0001:00002c34       __local_stdio_scanf_options 0000000180003c34 f i MSVCRT:default_local_stdio_options.obj
 0001:00002c3c       __scrt_initialize_default_local_stdio_options 0000000180003c3c f   MSVCRT:default_local_stdio_options.obj
 0001:00002c58       __scrt_get_dyn_tls_init_callback 0000000180003c58 f   MSVCRT:dyn_tls_init.obj
 0001:00002c60       _RTC_Initialize            0000000180003c60 f   MSVCRT:initsect.obj
 0001:00002c9c       _RTC_Terminate             0000000180003c9c f   MSVCRT:initsect.obj
 0001:00002cd8       __isa_available_init       0000000180003cd8 f   MSVCRT:cpu_disp.obj
 0001:00002e84       _get_startup_argv_mode     0000000180003e84 f   MSVCRT:argv_mode.obj
 0001:00002e8c       __scrt_is_ucrt_dll_in_use  0000000180003e8c f   MSVCRT:ucrt_detection.obj
 0001:00002ea0       memcpy                     0000000180003ea0 f   vcruntime:VCRUNTIME140.dll
 0001:00002ea6       memset                     0000000180003ea6 f   vcruntime:VCRUNTIME140.dll
 0001:00002eac       strchr                     0000000180003eac f   vcruntime:VCRUNTIME140.dll
 0001:00002eb2       __C_specific_handler       0000000180003eb2 f   vcruntime:VCRUNTIME140.dll
 0001:00002eb8       __std_type_info_destroy_list 0000000180003eb8 f   vcruntime:VCRUNTIME140.dll
 0001:00002ebe       strcmp                     0000000180003ebe f   ucrt:api-ms-win-crt-string-l1-1-0.dll
 0001:00002ec4       strlen                     0000000180003ec4 f   ucrt:api-ms-win-crt-string-l1-1-0.dll
 0001:00002eca       _initterm                  0000000180003eca f   ucrt:api-ms-win-crt-runtime-l1-1-0.dll
 0001:00002ed0       _initterm_e                0000000180003ed0 f   ucrt:api-ms-win-crt-runtime-l1-1-0.dll
 0001:00002ed6       _seh_filter_dll            0000000180003ed6 f   ucrt:api-ms-win-crt-runtime-l1-1-0.dll
 0001:00002edc       _configure_narrow_argv     0000000180003edc f   ucrt:api-ms-win-crt-runtime-l1-1-0.dll
 0001:00002ee2       _initialize_narrow_environment 0000000180003ee2 f   ucrt:api-ms-win-crt-runtime-l1-1-0.dll
 0001:00002ee8       _initialize_onexit_table   0000000180003ee8 f   ucrt:api-ms-win-crt-runtime-l1-1-0.dll
 0001:00002eee       _register_onexit_function  0000000180003eee f   ucrt:api-ms-win-crt-runtime-l1-1-0.dll
 0001:00002ef4       _execute_onexit_table      0000000180003ef4 f   ucrt:api-ms-win-crt-runtime-l1-1-0.dll
 0001:00002efa       _crt_atexit                0000000180003efa f   ucrt:api-ms-win-crt-runtime-l1-1-0.dll
 0001:00002f00       _cexit                     0000000180003f00 f   ucrt:api-ms-win-crt-runtime-l1-1-0.dll
 0001:00002f08       __acrt_initialize          0000000180003f08 f   MSVCRT:ucrt_stubs.obj
 0001:00002f08       __acrt_thread_attach       0000000180003f08 f   MSVCRT:ucrt_stubs.obj
 0001:00002f08       __acrt_thread_detach       0000000180003f08 f   MSVCRT:ucrt_stubs.obj
 0001:00002f08       __acrt_uninitialize        0000000180003f08 f   MSVCRT:ucrt_stubs.obj
 0001:00002f08       __acrt_uninitialize_critical 0000000180003f08 f   MSVCRT:ucrt_stubs.obj
 0001:00002f08       __scrt_stub_for_acrt_initialize 0000000180003f08 f   MSVCRT:ucrt_stubs.obj
 0001:00002f08       __scrt_stub_for_acrt_thread_attach 0000000180003f08 f   MSVCRT:ucrt_stubs.obj
 0001:00002f08       __scrt_stub_for_acrt_thread_detach 0000000180003f08 f   MSVCRT:ucrt_stubs.obj
 0001:00002f08       __scrt_stub_for_acrt_uninitialize 0000000180003f08 f   MSVCRT:ucrt_stubs.obj
 0001:00002f08       __scrt_stub_for_acrt_uninitialize_critical 0000000180003f08 f   MSVCRT:ucrt_stubs.obj
 0001:00002f08       __vcrt_initialize          0000000180003f08 f   MSVCRT:ucrt_stubs.obj
 0001:00002f08       __vcrt_thread_attach       0000000180003f08 f   MSVCRT:ucrt_stubs.obj
 0001:00002f08       __vcrt_thread_detach       0000000180003f08 f   MSVCRT:ucrt_stubs.obj
 0001:00002f08       __vcrt_uninitialize        0000000180003f08 f   MSVCRT:ucrt_stubs.obj
 0001:00002f08       __vcrt_uninitialize_critical 0000000180003f08 f   MSVCRT:ucrt_stubs.obj
 0001:00002f0c       __scrt_stub_for_is_c_termination_complete 0000000180003f0c f   MSVCRT:ucrt_stubs.obj
 0001:00002f0c       _is_c_termination_complete 0000000180003f0c f   MSVCRT:ucrt_stubs.obj
 0001:00002f20       _guard_dispatch_icall_nop  0000000180003f20 f   MSVCRT:guard_dispatch.obj
 0001:00002f40       _guard_xfg_dispatch_icall_nop 0000000180003f40 f   MSVCRT:guard_xfg_dispatch.obj
 0002:00000000       __imp_RtlCaptureContext    0000000180004000     kernel32:KERNEL32.dll
 0002:00000008       __imp_RtlLookupFunctionEntry 0000000180004008     kernel32:KERNEL32.dll
 0002:00000010       __imp_RtlVirtualUnwind     0000000180004010     kernel32:KERNEL32.dll
 0002:00000018       __imp_UnhandledExceptionFilter 0000000180004018     kernel32:KERNEL32.dll
 0002:00000020       __imp_SetUnhandledExceptionFilter 0000000180004020     kernel32:KERNEL32.dll
 0002:00000028       __imp_GetCurrentProcess    0000000180004028     kernel32:KERNEL32.dll
 0002:00000030       __imp_TerminateProcess     0000000180004030     kernel32:KERNEL32.dll
 0002:00000038       __imp_IsProcessorFeaturePresent 0000000180004038     kernel32:KERNEL32.dll
 0002:00000040       __imp_CloseHandle          0000000180004040     kernel32:KERNEL32.dll
 0002:00000048       __imp_InitializeCriticalSectionAndSpinCount 0000000180004048     kernel32:KERNEL32.dll
 0002:00000050       __imp_DeleteCriticalSection 0000000180004050     kernel32:KERNEL32.dll
 0002:00000058       __imp_CreateEventW         0000000180004058     kernel32:KERNEL32.dll
 0002:00000060       __imp_GetModuleHandleW     0000000180004060     kernel32:KERNEL32.dll
 0002:00000068       __imp_GetProcAddress       0000000180004068     kernel32:KERNEL32.dll
 0002:00000070       __imp_IsDebuggerPresent    0000000180004070     kernel32:KERNEL32.dll
 0002:00000078       __imp_QueryPerformanceCounter 0000000180004078     kernel32:KERNEL32.dll
 0002:00000080       __imp_GetCurrentProcessId  0000000180004080     kernel32:KERNEL32.dll
 0002:00000088       __imp_GetCurrentThreadId   0000000180004088     kernel32:KERNEL32.dll
 0002:00000090       __imp_GetSystemTimeAsFileTime 0000000180004090     kernel32:KERNEL32.dll
 0002:00000098       __imp_DisableThreadLibraryCalls 0000000180004098     kernel32:KERNEL32.dll
 0002:000000a0       __imp_InitializeSListHead  00000001800040a0     kernel32:KERNEL32.dll
 0002:000000a8       \177KERNEL32_NULL_THUNK_DATA 00000001800040a8     kernel32:KERNEL32.dll
 0002:000000b0       __imp_memcpy               00000001800040b0     vcruntime:VCRUNTIME140.dll
 0002:000000b8       __imp_memset               00000001800040b8     vcruntime:VCRUNTIME140.dll
 0002:000000c0       __imp_strchr               00000001800040c0     vcruntime:VCRUNTIME140.dll
 0002:000000c8       __imp___C_specific_handler 00000001800040c8     vcruntime:VCRUNTIME140.dll
 0002:000000d0       __imp___std_type_info_destroy_list 00000001800040d0     vcruntime:VCRUNTIME140.dll
 0002:000000d8       \177VCRUNTIME140_NULL_THUNK_DATA 00000001800040d8     vcruntime:VCRUNTIME140.dll
 0002:000000e0       __imp__errno               00000001800040e0     ucrt:api-ms-win-crt-runtime-l1-1-0.dll
 0002:000000e8       __imp_exit                 00000001800040e8     ucrt:api-ms-win-crt-runtime-l1-1-0.dll
 0002:000000f0       __imp__cexit               00000001800040f0     ucrt:api-ms-win-crt-runtime-l1-1-0.dll
 0002:000000f8       __imp__crt_atexit          00000001800040f8     ucrt:api-ms-win-crt-runtime-l1-1-0.dll
 0002:00000100       __imp__execute_onexit_table 0000000180004100     ucrt:api-ms-win-crt-runtime-l1-1-0.dll
 0002:00000108       __imp__register_onexit_function 0000000180004108     ucrt:api-ms-win-crt-runtime-l1-1-0.dll
 0002:00000110       __imp__initialize_onexit_table 0000000180004110     ucrt:api-ms-win-crt-runtime-l1-1-0.dll
 0002:00000118       __imp__initialize_narrow_environment 0000000180004118     ucrt:api-ms-win-crt-runtime-l1-1-0.dll
 0002:00000120       __imp__configure_narrow_argv 0000000180004120     ucrt:api-ms-win-crt-runtime-l1-1-0.dll
 0002:00000128       __imp__seh_filter_dll      0000000180004128     ucrt:api-ms-win-crt-runtime-l1-1-0.dll
 0002:00000130       __imp__initterm_e          0000000180004130     ucrt:api-ms-win-crt-runtime-l1-1-0.dll
 0002:00000138       __imp__initterm            0000000180004138     ucrt:api-ms-win-crt-runtime-l1-1-0.dll
 0002:00000140       \177api-ms-win-crt-runtime-l1-1-0_NULL_THUNK_DATA 0000000180004140     ucrt:api-ms-win-crt-runtime-l1-1-0.dll
 0002:00000148       __imp___acrt_iob_func      0000000180004148     ucrt:api-ms-win-crt-stdio-l1-1-0.dll
 0002:00000150       __imp_fflush               0000000180004150     ucrt:api-ms-win-crt-stdio-l1-1-0.dll
 0002:00000158       __imp___stdio_common_vsprintf 0000000180004158     ucrt:api-ms-win-crt-stdio-l1-1-0.dll
 0002:00000160       __imp___stdio_common_vfprintf 0000000180004160     ucrt:api-ms-win-crt-stdio-l1-1-0.dll
 0002:00000168       \177api-ms-win-crt-stdio-l1-1-0_NULL_THUNK_DATA 0000000180004168     ucrt:api-ms-win-crt-stdio-l1-1-0.dll
 0002:00000170       __imp_strcmp               0000000180004170     ucrt:api-ms-win-crt-string-l1-1-0.dll
 0002:00000178       __imp__strdup              0000000180004178     ucrt:api-ms-win-crt-string-l1-1-0.dll
 0002:00000178       __imp_strdup               0000000180004178     ucrt:api-ms-win-crt-string-l1-1-0.dll
 0002:00000180       __imp_strlen               0000000180004180     ucrt:api-ms-win-crt-string-l1-1-0.dll
 0002:00000188       __imp_strncpy              0000000180004188     ucrt:api-ms-win-crt-string-l1-1-0.dll
 0002:00000190       \177api-ms-win-crt-string-l1-1-0_NULL_THUNK_DATA 0000000180004190     ucrt:api-ms-win-crt-string-l1-1-0.dll
 0002:00000198       __guard_check_icall_fptr   0000000180004198     MSVCRT:guard_support.obj
 0002:000001a0       __guard_xfg_check_icall_fptr 00000001800041a0     MSVCRT:guard_support.obj
 0002:000001a8       __guard_dispatch_icall_fptr 00000001800041a8     MSVCRT:guard_support.obj
 0002:000001b0       __guard_xfg_dispatch_icall_fptr 00000001800041b0     MSVCRT:guard_support.obj
 0002:000001b8       __guard_xfg_table_dispatch_icall_fptr 00000001800041b8     MSVCRT:guard_support.obj
 0002:000001c0       __castguard_check_failure_os_handled_fptr 00000001800041c0     MSVCRT:guard_support.obj
 0002:000001c8       __guard_memcpy_fptr        00000001800041c8     vcruntime:softmemtag.obj
 0002:000001d0       __xc_a                     00000001800041d0     MSVCRT:initializers.obj
 0002:000001d8       __xc_z                     00000001800041d8     MSVCRT:initializers.obj
 0002:000001e0       __xi_a                     00000001800041e0     MSVCRT:initializers.obj
 0002:000001f0       __xi_z                     00000001800041f0     MSVCRT:initializers.obj
 0002:000001f8       __xl_a                     00000001800041f8     MSVCRT:tlssup.obj
 0002:00000200       __xl_z                     0000000180004200     MSVCRT:tlssup.obj
 0002:00000208       __xp_a                     0000000180004208     MSVCRT:initializers.obj
 0002:00000210       __xp_z                     0000000180004210     MSVCRT:initializers.obj
 0002:00000218       __xt_a                     0000000180004218     MSVCRT:initializers.obj
 0002:00000220       __xt_z                     0000000180004220     MSVCRT:initializers.obj
 0002:00000230       g_refKindStr               0000000180004230     libsetlocal004.obj
 0002:000003e0       ??_C@_09BPLDFGCI@unknown_0@ 00000001800043e0     libsetlocal004.obj
 0002:000003f0       ??_C@_0BL@FPNMECJD@JVMTI_HEAP_REFERENCE_CLASS@ 00000001800043f0     libsetlocal004.obj
 0002:00000410       ??_C@_0BL@FKGKKLNM@JVMTI_HEAP_REFERENCE_FIELD@ 0000000180004410     libsetlocal004.obj
 0002:00000430       ??_C@_0CD@CAEHCFJF@JVMTI_HEAP_REFERENCE_ARRAY_ELEM@ 0000000180004430     libsetlocal004.obj
 0002:00000458       ??_C@_0CC@DNEBMCNK@JVMTI_HEAP_REFERENCE_CLASS_LOAD@ 0000000180004458     libsetlocal004.obj
 0002:00000480       ??_C@_0BN@CJMIPEBB@JVMTI_HEAP_REFERENCE_SIGNERS@ 0000000180004480     libsetlocal004.obj
 0002:000004a0       ??_C@_0CH@HBOIDPEB@JVMTI_HEAP_REFERENCE_PROTECTION@ 00000001800044a0     libsetlocal004.obj
 0002:000004c8       ??_C@_0BP@MDKGDGKL@JVMTI_HEAP_REFERENCE_INTERFACE@ 00000001800044c8     libsetlocal004.obj
 0002:000004e8       ??_C@_0CC@JJMIHNJH@JVMTI_HEAP_REFERENCE_STATIC_FIE@ 00000001800044e8     libsetlocal004.obj
 0002:00000510       ??_C@_0CD@IDHEEGID@JVMTI_HEAP_REFERENCE_CONSTANT_P@ 0000000180004510     libsetlocal004.obj
 0002:00000538       ??_C@_0CA@EFFCHNG@JVMTI_HEAP_REFERENCE_SUPERCLASS@ 0000000180004538     libsetlocal004.obj
 0002:00000558       ??_C@_0L@PCDFHGCJ@unknown_11@ 0000000180004558     libsetlocal004.obj
 0002:00000568       ??_C@_0L@NJBICFOK@unknown_12@ 0000000180004568     libsetlocal004.obj
 0002:00000578       ??_C@_0L@MAADBEKL@unknown_13@ 0000000180004578     libsetlocal004.obj
 0002:00000588       ??_C@_0L@IPECICGM@unknown_14@ 0000000180004588     libsetlocal004.obj
 0002:00000598       ??_C@_0L@JGFJLDCN@unknown_15@ 0000000180004598     libsetlocal004.obj
 0002:000005a8       ??_C@_0L@LNHEOAOO@unknown_16@ 00000001800045a8     libsetlocal004.obj
 0002:000005b8       ??_C@_0L@KEGPNBKP@unknown_17@ 00000001800045b8     libsetlocal004.obj
 0002:000005c8       ??_C@_0L@CDPHMNGA@unknown_18@ 00000001800045c8     libsetlocal004.obj
 0002:000005d8       ??_C@_0L@DKOMPMCB@unknown_19@ 00000001800045d8     libsetlocal004.obj
 0002:000005e8       ??_C@_0L@OJGIPJDB@unknown_20@ 00000001800045e8     libsetlocal004.obj
 0002:000005f8       ??_C@_0CA@KAOFNDEM@JVMTI_HEAP_REFERENCE_JNI_GLOBAL@ 00000001800045f8     libsetlocal004.obj
 0002:00000618       ??_C@_0CC@HPFAJBK@JVMTI_HEAP_REFERENCE_SYSTEM_CLA@ 0000000180004618     libsetlocal004.obj
 0002:00000640       ??_C@_0BN@FDEGFOHC@JVMTI_HEAP_REFERENCE_MONITOR@ 0000000180004640     libsetlocal004.obj
 0002:00000660       ??_C@_0CB@HKIBCMAJ@JVMTI_HEAP_REFERENCE_STACK_LOCA@ 0000000180004660     libsetlocal004.obj
 0002:00000688       ??_C@_0BP@EAACMMOE@JVMTI_HEAP_REFERENCE_JNI_LOCAL@ 0000000180004688     libsetlocal004.obj
 0002:000006a8       ??_C@_0BM@IJDEOGOE@JVMTI_HEAP_REFERENCE_THREAD@ 00000001800046a8     libsetlocal004.obj
 0002:000006c8       ??_C@_0BL@EDGPPKC@JVMTI_HEAP_REFERENCE_OTHER@ 00000001800046c8     libsetlocal004.obj
 0002:000006e4       ??_C@_04BCJPDBDA@Code@     00000001800046e4     libsetlocal004.obj
 0002:000006f0       ??_C@_0BA@OCLMCFKC@LineNumberTable@ 00000001800046f0     libsetlocal004.obj
 0002:00000700       ??_C@_0BD@CPAEPILC@LocalVariableTable@ 0000000180004700     libsetlocal004.obj
 0002:00000718       ??_C@_0BH@NMBDNHBD@LocalVariableTypeTable@ 0000000180004718     libsetlocal004.obj
 0002:00000730       ??_C@_0O@HIHEEDNJ@StackMapTable@ 0000000180004730     libsetlocal004.obj
 0002:00000740       ??_C@_0L@HCDIAMJG@?9?5?$CFs?0?5?$CFd?3?5@ 0000000180004740     libsetlocal004.obj
 0002:00000750       ??_C@_0JI@HLPECLFI@?$CD?5?4?4?4?6?$CD?5ERROR?3?5too?5many?5complai@ 0000000180004750     libsetlocal004.obj
 0002:000007f0       ??_C@_0ED@JNEKCCOB@The?5following?5fake?5exception?5st@ 00000001800047f0     libsetlocal004.obj
 0002:00000838       ??_C@_0CN@FCNMDFBH@nsk?4share?4Fake_Exception_for_RU@ 0000000180004838     libsetlocal004.obj
 0002:00000868       ??_C@_08PGFFNAEI@?$CI?$CFs?3?$CFd?$CJ?5@ 0000000180004868     libsetlocal004.obj
 0002:00000878       ??_C@_0DP@IENMAEGI@s?2test?2hotspot?2jtreg?2vmTestbase@ 0000000180004878     libsetlocal004.obj
 0002:000008b8       ??_C@_0BL@NDJLFFJB@?7at?5nsk_lvcomplain?$CI?$CFs?3?$CFd?$CJ?6@ 00000001800048b8     libsetlocal004.obj
 0002:000008d8       ??_C@_0BC@JOOKAFKF@?$CD?5ERROR?3?5?$CFs?0?5?$CFd?3?5@ 00000001800048d8     libsetlocal004.obj
 0002:000008f0       ??_C@_09KJEAHMEH@?$CD?5ERROR?3?5@ 00000001800048f0     libsetlocal004.obj
 0002:000008fc       ??_C@_02GPIOPFAK@?$DO?$DO@ 00000001800048fc     libsetlocal004.obj
 0002:00000900       ??_C@_02FODMEDOG@?$DM?$DM@ 0000000180004900     libsetlocal004.obj
 0002:00000904       ??_C@_02DJGKEECL@?4?4@     0000000180004904     libsetlocal004.obj
 0002:00000908       ??_C@_0O@CJPGJOAF@?9?5?$CFs?0?5?$CFd?3?5?$CFs?5@ 0000000180004908     libsetlocal004.obj
 0002:00000918       ??_C@_0CB@IAKPDOIC@?$CD?5?5?5verified?5assertion?5is?5FALSE@ 0000000180004918     libsetlocal004.obj
 0002:00000940       ??_C@_0CO@LGONDEPD@stdout?3?5fflush?5failed?5?9?5err?$DN?$CFd?5@ 0000000180004940     libsetlocal004.obj
 0002:00000970       ??_C@_0CO@KBGKJPBD@stderr?3?5fflush?5failed?5?9?5err?$DN?$CFd?5@ 0000000180004970     libsetlocal004.obj
 0002:000009a0       ??_C@_0BB@JCNMKLLK@JVMTI_ERROR_NONE@ 00000001800049a0     libsetlocal004.obj
 0002:000009b8       ??_C@_0BL@LDIMKLPH@JVMTI_ERROR_INVALID_THREAD@ 00000001800049b8     libsetlocal004.obj
 0002:000009d8       ??_C@_0CB@PJFPAIKJ@JVMTI_ERROR_INVALID_THREAD_GROU@ 00000001800049d8     libsetlocal004.obj
 0002:00000a00       ??_C@_0BN@LLMKHMNF@JVMTI_ERROR_INVALID_PRIORITY@ 0000000180004a00     libsetlocal004.obj
 0002:00000a20       ??_C@_0CB@MBOFKAGB@JVMTI_ERROR_THREAD_NOT_SUSPENDE@ 0000000180004a20     libsetlocal004.obj
 0002:00000a48       ??_C@_0BN@FABOLPBI@JVMTI_ERROR_THREAD_SUSPENDED@ 0000000180004a48     libsetlocal004.obj
 0002:00000a68       ??_C@_0BN@FDGNOBJM@JVMTI_ERROR_THREAD_NOT_ALIVE@ 0000000180004a68     libsetlocal004.obj
 0002:00000a88       ??_C@_0BL@GOBIFKNJ@JVMTI_ERROR_INVALID_OBJECT@ 0000000180004a88     libsetlocal004.obj
 0002:00000aa8       ??_C@_0BK@FCMAJPPC@JVMTI_ERROR_INVALID_CLASS@ 0000000180004aa8     libsetlocal004.obj
 0002:00000ac8       ??_C@_0BP@IKLLBKEB@JVMTI_ERROR_CLASS_NOT_PREPARED@ 0000000180004ac8     libsetlocal004.obj
 0002:00000ae8       ??_C@_0BN@KLPPLKG@JVMTI_ERROR_INVALID_METHODID@ 0000000180004ae8     libsetlocal004.obj
 0002:00000b08       ??_C@_0BN@BCEKOKND@JVMTI_ERROR_INVALID_LOCATION@ 0000000180004b08     libsetlocal004.obj
 0002:00000b28       ??_C@_0BM@DFDGPME@JVMTI_ERROR_INVALID_FIELDID@ 0000000180004b28     libsetlocal004.obj
 0002:00000b48       ??_C@_0BL@NELIEPEC@JVMTI_ERROR_NO_MORE_FRAMES@ 0000000180004b48     libsetlocal004.obj
 0002:00000b68       ??_C@_0BJ@BDBECFDM@JVMTI_ERROR_OPAQUE_FRAME@ 0000000180004b68     libsetlocal004.obj
 0002:00000b88       ??_C@_0BK@MIIFNLOB@JVMTI_ERROR_TYPE_MISMATCH@ 0000000180004b88     libsetlocal004.obj
 0002:00000ba8       ??_C@_0BJ@HPCAOILC@JVMTI_ERROR_INVALID_SLOT@ 0000000180004ba8     libsetlocal004.obj
 0002:00000bc8       ??_C@_0BG@CHILOPNI@JVMTI_ERROR_DUPLICATE@ 0000000180004bc8     libsetlocal004.obj
 0002:00000be0       ??_C@_0BG@DIEMLHKM@JVMTI_ERROR_NOT_FOUND@ 0000000180004be0     libsetlocal004.obj
 0002:00000bf8       ??_C@_0BM@NHMCKHOB@JVMTI_ERROR_INVALID_MONITOR@ 0000000180004bf8     libsetlocal004.obj
 0002:00000c18       ??_C@_0BO@PPEDAJGL@JVMTI_ERROR_NOT_MONITOR_OWNER@ 0000000180004c18     libsetlocal004.obj
 0002:00000c38       ??_C@_0BG@FCAIPEID@JVMTI_ERROR_INTERRUPT@ 0000000180004c38     libsetlocal004.obj
 0002:00000c50       ??_C@_0CB@EGDBNKOI@JVMTI_ERROR_INVALID_CLASS_FORMA@ 0000000180004c50     libsetlocal004.obj
 0002:00000c78       ??_C@_0CG@DGKOGIAL@JVMTI_ERROR_CIRCULAR_CLASS_DEFI@ 0000000180004c78     libsetlocal004.obj
 0002:00000ca0       ??_C@_0BP@ICEALPKC@JVMTI_ERROR_FAILS_VERIFICATION@ 0000000180004ca0     libsetlocal004.obj
 0002:00000cc0       ??_C@_0DC@JDACLMIO@JVMTI_ERROR_UNSUPPORTED_REDEFIN@ 0000000180004cc0     libsetlocal004.obj
 0002:00000cf8       ??_C@_0DE@GKDKNOMJ@JVMTI_ERROR_UNSUPPORTED_REDEFIN@ 0000000180004cf8     libsetlocal004.obj
 0002:00000d30       ??_C@_0BO@LAFKIOG@JVMTI_ERROR_INVALID_TYPESTATE@ 0000000180004d30     libsetlocal004.obj
 0002:00000d50       ??_C@_0DH@INDGCLLB@JVMTI_ERROR_UNSUPPORTED_REDEFIN@ 0000000180004d50     libsetlocal004.obj
 0002:00000d88       ??_C@_0DE@NHEOMMGI@JVMTI_ERROR_UNSUPPORTED_REDEFIN@ 0000000180004d88     libsetlocal004.obj
 0002:00000dc0       ??_C@_0CA@EKPNJOEP@JVMTI_ERROR_UNSUPPORTED_VERSION@ 0000000180004dc0     libsetlocal004.obj
 0002:00000de0       ??_C@_0BN@OFFMAHHL@JVMTI_ERROR_NAMES_DONT_MATCH@ 0000000180004de0     libsetlocal004.obj
 0002:00000e00       ??_C@_0DN@HHBBLAKE@JVMTI_ERROR_UNSUPPORTED_REDEFIN@ 0000000180004e00     libsetlocal004.obj
 0002:00000e40       ??_C@_0DO@HMBGBGNA@JVMTI_ERROR_UNSUPPORTED_REDEFIN@ 0000000180004e40     libsetlocal004.obj
 0002:00000e80       ??_C@_0BP@PBECGKHJ@JVMTI_ERROR_UNMODIFIABLE_CLASS@ 0000000180004e80     libsetlocal004.obj
 0002:00000ea0       ??_C@_0BK@CANILEHF@JVMTI_ERROR_NOT_AVAILABLE@ 0000000180004ea0     libsetlocal004.obj
 0002:00000ec0       ??_C@_0CE@INJKMEFK@JVMTI_ERROR_MUST_POSSESS_CAPABI@ 0000000180004ec0     libsetlocal004.obj
 0002:00000ee8       ??_C@_0BJ@LBFPFPDM@JVMTI_ERROR_NULL_POINTER@ 0000000180004ee8     libsetlocal004.obj
 0002:00000f08       ??_C@_0BP@CHJPNNEM@JVMTI_ERROR_ABSENT_INFORMATION@ 0000000180004f08     libsetlocal004.obj
 0002:00000f28       ??_C@_0BP@OMFMNLC@JVMTI_ERROR_INVALID_EVENT_TYPE@ 0000000180004f28     libsetlocal004.obj
 0002:00000f48       ??_C@_0BN@BIBNPHHO@JVMTI_ERROR_ILLEGAL_ARGUMENT@ 0000000180004f48     libsetlocal004.obj
 0002:00000f68       ??_C@_0BK@KKNDHDCE@JVMTI_ERROR_NATIVE_METHOD@ 0000000180004f68     libsetlocal004.obj
 0002:00000f88       ??_C@_0BK@PMKCFHAE@JVMTI_ERROR_OUT_OF_MEMORY@ 0000000180004f88     libsetlocal004.obj
 0002:00000fa8       ??_C@_0BK@NNJBDMNB@JVMTI_ERROR_ACCESS_DENIED@ 0000000180004fa8     libsetlocal004.obj
 0002:00000fc8       ??_C@_0BI@GHECLMNC@JVMTI_ERROR_WRONG_PHASE@ 0000000180004fc8     libsetlocal004.obj
 0002:00000fe0       ??_C@_0BF@OLIHJOII@JVMTI_ERROR_INTERNAL@ 0000000180004fe0     libsetlocal004.obj
 0002:00000ff8       ??_C@_0BO@EOHGKJHI@JVMTI_ERROR_UNATTACHED_THREAD@ 0000000180004ff8     libsetlocal004.obj
 0002:00001018       ??_C@_0CA@LKHFDACL@JVMTI_ERROR_INVALID_ENVIRONMENT@ 0000000180005018     libsetlocal004.obj
 0002:00001038       ??_C@_0BA@MMFHLOKK@?$DMunknown?5error?$DO@ 0000000180005038     libsetlocal004.obj
 0002:00001048       ??_C@_0CF@CBHOKDB@throwable?5?$DN?5jni?9?$DOExceptionOccur@ 0000000180005048     libsetlocal004.obj
 0002:00001070       ??_C@_03OFAPEBGM@?$CFs?6@  0000000180005070     libsetlocal004.obj
 0002:00001078       ??_C@_0DM@LPIGEGNJ@s?2test?2hotspot?2jtreg?2vmTestbase@ 0000000180005078     libsetlocal004.obj
 0002:000010b8       ??_C@_0CC@NFCNPEPK@Exception?5in?5JNI?5call?5?$CIcleared?$CJ@ 00000001800050b8     libsetlocal004.obj
 0002:000010e0       ??_C@_0BJ@IBAKFIKF@jni?9?$DOExceptionDescribe?$CI?$CJ@ 00000001800050e0     libsetlocal004.obj
 0002:00001100       ??_C@_0BG@GGKALKMH@jni?9?$DOExceptionClear?$CI?$CJ@ 0000000180005100     libsetlocal004.obj
 0002:00001118       ??_C@_0CF@JMGFGJLJ@?$CD?5?5?5verified?5JNI?5assertion?5is?5F@ 0000000180005118     libsetlocal004.obj
 0002:00001140       ??_C@_0CB@MLNJNCLJ@?5?5jvmti?5error?3?5code?$DN?$CFd?0?5name?$DN?$CFs@ 0000000180005140     libsetlocal004.obj
 0002:00001168       ??_C@_0CD@OHBGDKMK@?$CD?5?5?5jvmti?5error?3?5code?$DN?$CFd?0?5name?$DN@ 0000000180005168     libsetlocal004.obj
 0002:00001190       ??_C@_0CG@JNNCGPHB@?$CD?5?5?5error?5expected?3?5code?$DN?$CFd?0?5na@ 0000000180005190     libsetlocal004.obj
 0002:000011c0       ??_C@_0EB@IMGKPCGE@?$CIstr_obj?5?$DN?5jni?9?$DONewStringUTF?$CIco@ 00000001800051c0     libsetlocal004.obj
 0002:00001210       ??_C@_0EA@HFOGGBCC@s?2test?2hotspot?2jtreg?2vmTestbase@ 0000000180005210     libsetlocal004.obj
 0002:00001250       ??_C@_0CO@HJKAMPK@?$CIGetFrameLocation?$CJ?5unexpected?5e@ 0000000180005250     libsetlocal004.obj
 0002:00001280       ??_C@_05KKCIMGE@error@     0000000180005280     libsetlocal004.obj
 0002:00001288       ??_C@_0CJ@JACLEAA@Test?5failed?5by?5setFailStatus?$CI?$CJ?4@ 0000000180005288     libsetlocal004.obj
 0002:000012c0       ??_C@_0EA@PNBCDMOA@s?2test?2hotspot?2jtreg?2vmTestbase@ 00000001800052c0     libsetlocal004.obj
 0002:00001300       ??_C@_0DI@ILAHDLMP@?$CI?$CKagentThreadProc?$CJ?$CIjvmti_env?0?5a@ 0000000180005300     libsetlocal004.obj
 0002:00001338       ??_C@_0BD@KDBALNLB@JVMTI?5agent?5thread@ 0000000180005338     libsetlocal004.obj
 0002:00001350       ??_C@_0BB@NOKBFPFO@java?1lang?1Thread@ 0000000180005350     libsetlocal004.obj
 0002:00001364       ??_C@_06FALKBLGB@?$DMinit?$DO@ 0000000180005364     libsetlocal004.obj
 0002:00001370       ??_C@_0BG@IKDDPPGD@?$CILjava?1lang?1String?$DL?$CJV@ 0000000180005370     libsetlocal004.obj
 0002:00001390       ??_C@_0EB@IFJBFEKC@?$CIthreadClass?5?$DN?5jni_env?9?$DOFindCla@ 0000000180005390     libsetlocal004.obj
 0002:000013e0       ??_C@_0GF@FGFIBKKL@?$CIthreadCtor?5?$DN?5jni_env?9?$DOGetMetho@ 00000001800053e0     libsetlocal004.obj
 0002:00001448       ??_C@_0DN@NCPDJLOG@?$CIthreadName?5?$DN?5jni_env?9?$DONewStrin@ 0000000180005448     libsetlocal004.obj
 0002:00001490       ??_C@_0FE@PFKODBGC@?$CIthreadObject?5?$DN?5jni_env?9?$DONewObj@ 0000000180005490     libsetlocal004.obj
 0002:000014f0       ??_C@_0ED@HOBAHHJI@?$CIthreadGlobalRef?5?$DN?5jni_env?9?$DONew@ 00000001800054f0     libsetlocal004.obj
 0002:00001540       ??_C@_0FN@HNJJAHFC@jvmti_env?9?$DORunAgentThread?$CIagent@ 0000000180005540     libsetlocal004.obj
 0002:000015a0       ??_C@_0EA@MOJDNKDF@Debuggee?5status?5sync?5aborted?5be@ 00000001800055a0     libsetlocal004.obj
 0002:000015e0       ??_C@_0EA@EEOEJAEN@status?5?$DN?5syncDebuggeeStatus?$CIjni@ 00000001800055e0     libsetlocal004.obj
 0002:00001620       ??_C@_0BL@JBCFNBMB@nsk_jvmti_resetAgentData?$CI?$CJ@ 0000000180005620     libsetlocal004.obj
 0002:00001640       ??_C@_0EL@LPBEELIP@s?2test?2hotspot?2jtreg?2vmTestbase@ 0000000180005640     libsetlocal004.obj
 0002:00001690       ??_C@_0CK@JDAMFDMJ@jvmti?9?$DOSetTag?$CIo?0?5tag?$CJ?5?$DN?$DN?5JVMTI_@ 0000000180005690     libsetlocal004.obj
 0002:000016c0       ??_C@_0CC@DAMNHKNI@Can?8t?5set?5tag?5?$CFli?5for?5object?5?$CFl@ 00000001800056c0     libsetlocal004.obj
 0002:000016e8       ??_C@_0DL@HAJPNKEF@jvmti?9?$DOGetObjectHashCode?$CIo?0?5?$CGha@ 00000001800056e8     libsetlocal004.obj
 0002:00001728       ??_C@_0BL@JFPIEOBF@Can?8t?5get?5hash?5object?5?$CFlx?6@ 0000000180005728     libsetlocal004.obj
 0002:00001748       ??_C@_0BG@DICPHBKN@setTag?3?5?$CF08x?5?$DM?9?5?$CF?53li@ 0000000180005748     libsetlocal004.obj
 0002:00001760       ??_C@_0DH@FCEEBDMJ@?$CIs?5?$DN?5jni?9?$DOGetStringUTFChars?$CIsIn@ 0000000180005760     libsetlocal004.obj
 0002:00001798       ??_C@_0BJ@OKKGHDCN@Can?8t?5get?5string?5at?5?$CF?$CDp?6@ 0000000180005798     libsetlocal004.obj
 0002:000017b8       ??_C@_0BP@EKFLGGFJ@Can?8t?5get?5string?5at?5?$CF?$CDp?3?5null?6@ 00000001800057b8     libsetlocal004.obj
 0002:000017d8       ??_C@_06ICODBHCL@?5?1?1?5?$CFs@ 00000001800057d8     libsetlocal004.obj
 0002:000017e0       ??_C@_0DB@KGFPLEGO@?$CIr?5?$DN?5jvmti?9?$DOGetTag?$CIo?0?5?$CGtag?$CJ?$CJ?5?$DN?$DN@ 00000001800057e0     libsetlocal004.obj
 0002:00001818       ??_C@_0CO@PDAGBCGJ@Can?8t?5GetTag?5for?5object?5?$CFlx?4?5Re@ 0000000180005818     libsetlocal004.obj
 0002:00001848       ??_C@_0CH@HPEODOHC@TEST_BUG?3?5Max?4?5number?5of?5refs?5r@ 0000000180005848     libsetlocal004.obj
 0002:00001870       ??_C@_0DI@PHFCABIM@?$CIr?5?$DN?5jvmti?9?$DOGetTag?$CIfrom?0?5?$CGtagFr@ 0000000180005870     libsetlocal004.obj
 0002:000018a8       ??_C@_0DI@MDEGFNKD@TEST_BUG?3?5Can?8t?5GetTag?5for?5obje@ 00000001800058a8     libsetlocal004.obj
 0002:000018e0       ??_C@_0DE@MLELJAHM@?$CIr?5?$DN?5jvmti?9?$DOGetTag?$CIto?0?5?$CGtagTo?$CJ?$CJ@ 00000001800058e0     libsetlocal004.obj
 0002:00001914       ??_C@_03GAEACAIP@?$CI?$CJV@ 0000000180005914     libsetlocal004.obj
 0002:00001918       ??_C@_05HHHBCPMM@?$CI?$CFs?$CJ?5@ 0000000180005918     libsetlocal004.obj
 0002:00001920       ??_C@_0EJ@FEJLMIEN@Error?3?5expected?3?5JVMTI_ERROR_TY@ 0000000180005920     libsetlocal004.obj
 0002:00001970       ??_C@_0BG@MMCFPIHA@?7?5?5?5?5actual?3?5?$CFs?5?$CI?$CFd?$CJ?6@ 0000000180005970     libsetlocal004.obj
 0002:00001988       ??_C@_0CL@GGLLOPOO@?$DO?$DO?$DO?5obtaining?5local?5variables?5m@ 0000000180005988     libsetlocal004.obj
 0002:000019b8       ??_C@_0DD@ELHIJBGO@?$CIGetLocalVariableTable?$CJ?5unexpec@ 00000001800059b8     libsetlocal004.obj
 0002:000019f0       ??_C@_0CD@NIDGFFEL@?$DO?$DO?$DO?5checking?5on?5type?5mismatch?5?4@ 00000001800059f0     libsetlocal004.obj
 0002:00001a14       ??_C@_01FMEDJKGI@o@        0000000180005a14     libsetlocal004.obj
 0002:00001a18       ??_C@_01KBJDNOO@i@         0000000180005a18     libsetlocal004.obj
 0002:00001a1c       ??_C@_01HHGOMJKL@l@        0000000180005a1c     libsetlocal004.obj
 0002:00001a20       ??_C@_01INIBCBCB@f@        0000000180005a20     libsetlocal004.obj
 0002:00001a24       ??_C@_01LPLHEDKD@d@        0000000180005a24     libsetlocal004.obj
 0002:00001a28       ??_C@_0O@BHPJPDFF@?$DO?$DO?$DO?5?4?4?4?5done?6@ 0000000180005a28     libsetlocal004.obj
 0002:00001a38       ??_C@_09OPJEJKBL@printdump@ 0000000180005a38     libsetlocal004.obj
 0002:00001a48       ??_C@_0CJ@KCDEKOCJ@Wrong?5result?5of?5a?5valid?5call?5to@ 0000000180005a48     libsetlocal004.obj
 0002:00001a78       ??_C@_0DG@LAJPGIIE@?$CIGetPotentialCapabilities?$CJ?5unex@ 0000000180005a78     libsetlocal004.obj
 0002:00001ab0       ??_C@_0CN@LKPEOJPO@?$CIAddCapabilities?$CJ?5unexpected?5er@ 0000000180005ab0     libsetlocal004.obj
 0002:00001ae0       ??_C@_0CN@BCCBOHCH@?$CIGetCapabilities?$CJ?5unexpected?5er@ 0000000180005ae0     libsetlocal004.obj
 0002:00001b10       ??_C@_0DH@IJEIPLEC@Warning?3?5access?5to?5local?5variab@ 0000000180005b10     libsetlocal004.obj
 0002:00001b48       ??_C@_0CP@IMINGNLL@?$CISetEventCallbacks?$CJ?5unexpected?5@ 0000000180005b48     libsetlocal004.obj
 0002:00001b78       ??_C@_0CO@FDBBPEKA@Warning?3?5Breakpoint?5event?5is?5no@ 0000000180005b78     libsetlocal004.obj
 0002:00001ba8       ??_C@_0CH@CDOJMNAO@JVMTI?5client?5was?5not?5properly?5l@ 0000000180005ba8     libsetlocal004.obj
 0002:00001bd0       ??_C@_0L@GIHILDI@checkPoint@ 0000000180005bd0     libsetlocal004.obj
 0002:00001be0       ??_C@_0CN@GIADEMBI@Cannot?5find?5Method?5ID?5for?5metho@ 0000000180005be0     libsetlocal004.obj
 0002:00001c10       ??_C@_0CC@GAODDEMK@Failed?5to?5SetBreakpoint?3?5?$CFs?5?$CI?$CFd@ 0000000180005c10     libsetlocal004.obj
 0002:00001c38       ??_C@_0CM@NEGFNKGE@Failed?5to?5enable?5BREAKPOINT?5eve@ 0000000180005c38     libsetlocal004.obj
 0002:00001c80       ??_C@_1EC@JIJBPKFM@?$AAa?$AAp?$AAi?$AA?9?$AAm?$AAs?$AA?9?$AAw?$AAi?$AAn?$AA?9?$AAc?$AAo?$AAr?$AAe@ 0000000180005c80     MSVCRT:thread_safe_statics.obj
 0002:00001cc8       ??_C@_1BK@MGMFAEKH@?$AAk?$AAe?$AAr?$AAn?$AAe?$AAl?$AA3?$AA2?$AA?4?$AAd?$AAl?$AAl@ 0000000180005cc8     MSVCRT:thread_safe_statics.obj
 0002:00001ce8       ??_C@_0BJ@JEBJOJFJ@SleepConditionVariableCS@ 0000000180005ce8     MSVCRT:thread_safe_statics.obj
 0002:00001d08       ??_C@_0BJ@PGPPEPCC@WakeAllConditionVariable@ 0000000180005d08     MSVCRT:thread_safe_statics.obj
 0002:00001d28       _pDefaultRawDllMain        0000000180005d28     MSVCRT:dll_dllmain.obj
 0002:00001d28       _pRawDllMain               0000000180005d28     MSVCRT:dll_dllmain.obj
 0002:00001d30       __xmm@ffffffffffffffffffffffffffffffff 0000000180005d30     MSVCRT:utility.obj
 0002:00001d40       _load_config_used          0000000180005d40     MSVCRT:loadcfg.obj
 0002:00001f00       _tls_used                  0000000180005f00     MSVCRT:tlssup.obj
 0002:00001f28       __volatile_metadata        0000000180005f28     <linker-defined>
 0002:000022e8       __rtc_iaa                  00000001800062e8     MSVCRT:initsect.obj
 0002:000022f0       __rtc_izz                  00000001800062f0     MSVCRT:initsect.obj
 0002:000022f8       __rtc_taa                  00000001800062f8     MSVCRT:initsect.obj
 0002:00002300       __rtc_tzz                  0000000180006300     MSVCRT:initsect.obj
 0002:00002308       _tls_start                 0000000180006308     MSVCRT:tlssup.obj
 0002:0000230c       _Init_thread_epoch         000000018000630c     MSVCRT:thread_safe_statics.obj
 0002:00002310       _tls_end                   0000000180006310     MSVCRT:tlssup.obj
 0002:000029f0       __IMPORT_DESCRIPTOR_KERNEL32 00000001800069f0     kernel32:KERNEL32.dll
 0002:00002a04       __IMPORT_DESCRIPTOR_VCRUNTIME140 0000000180006a04     vcruntime:VCRUNTIME140.dll
 0002:00002a18       __IMPORT_DESCRIPTOR_api-ms-win-crt-runtime-l1-1-0 0000000180006a18     ucrt:api-ms-win-crt-runtime-l1-1-0.dll
 0002:00002a2c       __IMPORT_DESCRIPTOR_api-ms-win-crt-stdio-l1-1-0 0000000180006a2c     ucrt:api-ms-win-crt-stdio-l1-1-0.dll
 0002:00002a40       __IMPORT_DESCRIPTOR_api-ms-win-crt-string-l1-1-0 0000000180006a40     ucrt:api-ms-win-crt-string-l1-1-0.dll
 0002:00002a54       __NULL_IMPORT_DESCRIPTOR   0000000180006a54     kernel32:KERNEL32.dll
 0003:00000030       _Init_global_epoch         0000000180008030     MSVCRT:thread_safe_statics.obj
 0003:00000040       __security_cookie          0000000180008040     MSVCRT:gs_cookie.obj
 0003:00000048       __security_cookie_complement 0000000180008048     MSVCRT:gs_cookie.obj
 0003:00000050       _fltused                   0000000180008050     MSVCRT:fltused.obj
 0003:00000054       __scrt_native_dllmain_reason 0000000180008054     MSVCRT:utility.obj
 0003:00000058       __isa_available            0000000180008058     MSVCRT:cpu_disp.obj
 0003:0000005c       __isa_enabled              000000018000805c     MSVCRT:cpu_disp.obj
 0003:00000060       __memset_fast_string_threshold 0000000180008060     MSVCRT:cpu_disp.obj
 0003:00000068       __memset_nt_threshold      0000000180008068     MSVCRT:cpu_disp.obj
 0003:00000070       __scrt_ucrt_dll_is_in_use  0000000180008070     MSVCRT:ucrt_stubs.obj
 0003:00000080       g_wrongHeapCallbacks       0000000180008080     libsetlocal004.obj
 0003:00000100       g_szTagInfo                0000000180008100     libsetlocal004.obj
 0003:00002040       g_tagFlags                 000000018000a040     libsetlocal004.obj
 0003:00002428       g_refsToVerifyCnt          000000018000a428     libsetlocal004.obj
 0003:0000242c       g_fakeUserData             000000018000a42c     libsetlocal004.obj
 0003:00002430       g_tagVisitCount            000000018000a430     libsetlocal004.obj
 0003:000033d0       g_refsToVerify             000000018000b3d0     libsetlocal004.obj
 0003:0001aad0       g_userDataError            0000000180022ad0     libsetlocal004.obj
 0003:0001adb8       ?_OptionsStorage@?1??__local_stdio_printf_options@@9@4_KA 0000000180022db8     libsetlocal004.obj
 0003:0001b378       _tls_index                 0000000180023378     MSVCRT:tlssup.obj
 0003:0001b380       __scrt_current_native_startup_state 0000000180023380     MSVCRT:utility.obj
 0003:0001b388       __scrt_native_startup_lock 0000000180023388     MSVCRT:utility.obj
 0003:0001b3c8       __scrt_debugger_hook_flag  00000001800233c8     MSVCRT:utility_desktop.obj
 0003:0001b3d0       ?__type_info_root_node@@3U__type_info_node@@A 00000001800233d0     MSVCRT:tncleanup.obj
 0003:0001b3e0       ?_OptionsStorage@?1??__local_stdio_scanf_options@@9@4_KA 00000001800233e0     MSVCRT:default_local_stdio_options.obj
 0003:0001b3e8       __favor                    00000001800233e8     MSVCRT:cpu_disp.obj
 0003:0001b3f0       __dyn_tls_init_callback    00000001800233f0     <common>

 entry point at        0001:00002630

 Static symbols

 0000:fffda000       .debug$S                   0000000180000000     setlocal004.exp
 0000:fffda000       .debug$S                   0000000180000000     vcruntime:VCRUNTIME140.dll
 0000:fffda000       .debug$S                   0000000180000000     vcruntime:VCRUNTIME140.dll
 0000:fffda000       .debug$S                   0000000180000000     vcruntime:VCRUNTIME140.dll
 0000:fffda000       .debug$S                   0000000180000000     vcruntime:VCRUNTIME140.dll
 0000:fffda000       .debug$S                   0000000180000000     vcruntime:VCRUNTIME140.dll
 0000:fffda000       .debug$S                   0000000180000000     vcruntime:VCRUNTIME140.dll
 0000:fffda000       .debug$S                   0000000180000000     vcruntime:VCRUNTIME140.dll
 0000:fffda000       .debug$S                   0000000180000000     ucrt:api-ms-win-crt-convert-l1-1-0.dll
 0002:ffffc000       .idata$6                   0000000180000000     ucrt:api-ms-win-crt-convert-l1-1-0.dll
 0000:fffda000       .debug$S                   0000000180000000     ucrt:api-ms-win-crt-heap-l1-1-0.dll
 0000:fffda000       .debug$S                   0000000180000000     ucrt:api-ms-win-crt-heap-l1-1-0.dll
 0000:fffda000       .debug$S                   0000000180000000     ucrt:api-ms-win-crt-heap-l1-1-0.dll
 0000:fffda000       .debug$S                   0000000180000000     ucrt:api-ms-win-crt-heap-l1-1-0.dll
 0002:ffffc000       .idata$6                   0000000180000000     ucrt:api-ms-win-crt-heap-l1-1-0.dll
 0000:fffda000       .debug$S                   0000000180000000     ucrt:api-ms-win-crt-runtime-l1-1-0.dll
 0000:fffda000       .debug$S                   0000000180000000     ucrt:api-ms-win-crt-runtime-l1-1-0.dll
 0000:fffda000       .debug$S                   0000000180000000     ucrt:api-ms-win-crt-runtime-l1-1-0.dll
 0000:fffda000       .debug$S                   0000000180000000     ucrt:api-ms-win-crt-runtime-l1-1-0.dll
 0000:fffda000       .debug$S                   0000000180000000     ucrt:api-ms-win-crt-runtime-l1-1-0.dll
 0000:fffda000       .debug$S                   0000000180000000     ucrt:api-ms-win-crt-runtime-l1-1-0.dll
 0000:fffda000       .debug$S                   0000000180000000     ucrt:api-ms-win-crt-runtime-l1-1-0.dll
 0000:fffda000       .debug$S                   0000000180000000     ucrt:api-ms-win-crt-runtime-l1-1-0.dll
 0000:fffda000       .debug$S                   0000000180000000     ucrt:api-ms-win-crt-runtime-l1-1-0.dll
 0000:fffda000       .debug$S                   0000000180000000     ucrt:api-ms-win-crt-runtime-l1-1-0.dll
 0000:fffda000       .debug$S                   0000000180000000     ucrt:api-ms-win-crt-runtime-l1-1-0.dll
 0000:fffda000       .debug$S                   0000000180000000     ucrt:api-ms-win-crt-runtime-l1-1-0.dll
 0000:fffda000       .debug$S                   0000000180000000     ucrt:api-ms-win-crt-runtime-l1-1-0.dll
 0000:fffda000       .debug$S                   0000000180000000     ucrt:api-ms-win-crt-runtime-l1-1-0.dll
 0000:fffda000       .debug$S                   0000000180000000     ucrt:api-ms-win-crt-runtime-l1-1-0.dll
 0000:fffda000       .debug$S                   0000000180000000     ucrt:api-ms-win-crt-runtime-l1-1-0.dll
 0000:fffda000       .debug$S                   0000000180000000     ucrt:api-ms-win-crt-stdio-l1-1-0.dll
 0000:fffda000       .debug$S                   0000000180000000     ucrt:api-ms-win-crt-stdio-l1-1-0.dll
 0000:fffda000       .debug$S                   0000000180000000     ucrt:api-ms-win-crt-stdio-l1-1-0.dll
 0000:fffda000       .debug$S                   0000000180000000     ucrt:api-ms-win-crt-stdio-l1-1-0.dll
 0000:fffda000       .debug$S                   0000000180000000     ucrt:api-ms-win-crt-stdio-l1-1-0.dll
 0000:fffda000       .debug$S                   0000000180000000     ucrt:api-ms-win-crt-stdio-l1-1-0.dll
 0000:fffda000       .debug$S                   0000000180000000     ucrt:api-ms-win-crt-stdio-l1-1-0.dll
 0000:fffda000       .debug$S                   0000000180000000     ucrt:api-ms-win-crt-stdio-l1-1-0.dll
 0000:fffda000       .debug$S                   0000000180000000     ucrt:api-ms-win-crt-stdio-l1-1-0.dll
 0000:fffda000       .debug$S                   0000000180000000     ucrt:api-ms-win-crt-stdio-l1-1-0.dll
 0000:fffda000       .debug$S                   0000000180000000     ucrt:api-ms-win-crt-string-l1-1-0.dll
 0000:fffda000       .debug$S                   0000000180000000     ucrt:api-ms-win-crt-string-l1-1-0.dll
 0000:fffda000       .debug$S                   0000000180000000     ucrt:api-ms-win-crt-string-l1-1-0.dll
 0000:fffda000       .debug$S                   0000000180000000     ucrt:api-ms-win-crt-string-l1-1-0.dll
 0000:fffda000       .debug$S                   0000000180000000     ucrt:api-ms-win-crt-string-l1-1-0.dll
 0000:fffda000       .debug$S                   0000000180000000     ucrt:api-ms-win-crt-string-l1-1-0.dll
 0000:fffda000       .debug$S                   0000000180000000     ucrt:api-ms-win-crt-string-l1-1-0.dll
 0000:fffda000       .debug$S                   0000000180000000     ucrt:api-ms-win-crt-string-l1-1-0.dll
 0000:fffda000       .debug$S                   0000000180000000     kernel32:KERNEL32.dll
 0000:fffda000       .debug$S                   0000000180000000     kernel32:KERNEL32.dll
 0000:fffda000       .debug$S                   0000000180000000     kernel32:KERNEL32.dll
 0000:fffda000       .debug$S                   0000000180000000     kernel32:KERNEL32.dll
 0000:fffda000       .debug$S                   0000000180000000     kernel32:KERNEL32.dll
 0000:fffda000       .debug$S                   0000000180000000     kernel32:KERNEL32.dll
 0000:fffda000       .debug$S                   0000000180000000     kernel32:KERNEL32.dll
 0000:fffda000       .debug$S                   0000000180000000     kernel32:KERNEL32.dll
 0000:fffda000       .debug$S                   0000000180000000     kernel32:KERNEL32.dll
 0000:fffda000       .debug$S                   0000000180000000     kernel32:KERNEL32.dll
 0000:fffda000       .debug$S                   0000000180000000     kernel32:KERNEL32.dll
 0000:fffda000       .debug$S                   0000000180000000     kernel32:KERNEL32.dll
 0000:fffda000       .debug$S                   0000000180000000     kernel32:KERNEL32.dll
 0000:fffda000       .debug$S                   0000000180000000     kernel32:KERNEL32.dll
 0000:fffda000       .debug$S                   0000000180000000     kernel32:KERNEL32.dll
 0000:fffda000       .debug$S                   0000000180000000     kernel32:KERNEL32.dll
 0000:fffda000       .debug$S                   0000000180000000     kernel32:KERNEL32.dll
 0000:fffda000       .debug$S                   0000000180000000     kernel32:KERNEL32.dll
 0000:fffda000       .debug$S                   0000000180000000     kernel32:KERNEL32.dll
 0000:fffda000       .debug$S                   0000000180000000     kernel32:KERNEL32.dll
 0000:fffda000       .debug$S                   0000000180000000     kernel32:KERNEL32.dll
 0000:fffda000       .debug$S                   0000000180000000     kernel32:KERNEL32.dll
 0000:fffda000       .debug$S                   0000000180000000     kernel32:KERNEL32.dll
 0000:fffda000       .debug$S                   0000000180000000     kernel32:KERNEL32.dll
 0000:fffda000       .debug$S                   0000000180000000     kernel32:KERNEL32.dll
 0000:fffda000       .debug$S                   0000000180000000     kernel32:KERNEL32.dll
 0000:fffda000       .debug$S                   0000000180000000     kernel32:KERNEL32.dll
 0000:fffda000       .debug$S                   0000000180000000     kernel32:KERNEL32.dll
 0001:000011e8       addRefToVerify             00000001800021e8 f   libsetlocal004.obj
 0001:00001254       agentThreadWrapper         0000000180002254 f   libsetlocal004.obj
 0001:000013c0       check_error                00000001800023c0 f   libsetlocal004.obj
 0001:000014a0       file_basename              00000001800024a0 f   libsetlocal004.obj
 0001:00001b0c       startAgentThreadWrapper    0000000180002b0c f   libsetlocal004.obj
 0001:00001e4c       syncDebuggeeStatus         0000000180002e4c f   libsetlocal004.obj
 0001:000020ec       capture_previous_context   00000001800030ec f   MSVCRT:gs_report.obj
 0001:00002160       ?__scrt_initialize_thread_safe_statics@@YAHXZ 0000000180003160 f   MSVCRT:thread_safe_statics.obj
 0001:00002230       ?__scrt_uninitialize_thread_safe_statics@@YAXXZ 0000000180003230 f   MSVCRT:thread_safe_statics.obj
 0001:000022e0       $$000000                   00000001800032e0     MSVCRT:amdsecgs.obj
 0001:00002310       ?dllmain_crt_dispatch@@YAHQEAUHINSTANCE__@@KQEAX@Z 0000000180003310 f   MSVCRT:dll_dllmain.obj
 0001:00002360       ?dllmain_crt_process_attach@@YAHQEAUHINSTANCE__@@QEAX@Z 0000000180003360 f   MSVCRT:dll_dllmain.obj
 0001:00002478       ?dllmain_crt_process_detach@@YAH_N@Z 0000000180003478 f   MSVCRT:dll_dllmain.obj
 0001:000024fc       ?dllmain_dispatch@@YAHQEAUHINSTANCE__@@KQEAX@Z 00000001800034fc f   MSVCRT:dll_dllmain.obj
 0001:00002f10       $$000000                   0000000180003f10     MSVCRT:guard_dispatch.obj
 0001:00002f30       $$000000                   0000000180003f30     MSVCRT:guard_xfg_dispatch.obj
 0001:00002f46       ?fin$0@?0??dllmain_crt_process_attach@@YAHQEAUHINSTANCE__@@QEAX@Z@4HA 0000000180003f46 f   MSVCRT:dll_dllmain.obj
 0001:00002f5d       ?fin$0@?0??dllmain_crt_process_detach@@YAH_N@Z@4HA 0000000180003f5d f   MSVCRT:dll_dllmain.obj
 0001:00002f76       ?fin$1@?0??dllmain_crt_process_detach@@YAH_N@Z@4HA 0000000180003f76 f   MSVCRT:dll_dllmain.obj
 0001:00002f8a       ?filt$0@?0??dllmain_dispatch@@YAHQEAUHINSTANCE__@@KQEAX@Z@4HA 0000000180003f8a f   MSVCRT:dll_dllmain.obj
 0001:00002fc0       __scrt_is_nonwritable_in_current_image$filt$0 0000000180003fc0 f   MSVCRT:utility.obj
 0002:000001e8       ?__scrt_initialize_tss_var@@3P6AHXZEA 00000001800041e8     MSVCRT:thread_safe_statics.obj
 0002:00000310       ?opcLengths@@3QBEB         0000000180004310     libsetlocal004.obj
 0002:00001c68       GS_ExceptionPointers       0000000180005c68     MSVCRT:gs_report.obj
 0002:00002318       $unwind$fprintf            0000000180006318     libsetlocal004.obj
 0002:00002324       $unwind$printf             0000000180006324     libsetlocal004.obj
 0002:00002330       $unwind$?NewObject@JNIEnv_@@QEAAPEAV_jobject@@PEAV_jclass@@PEAU_jmethodID@@ZZ 0000000180006330     libsetlocal004.obj
 0002:00002330       $unwind$nsk_lcomplain      0000000180006330     libsetlocal004.obj
 0002:00002330       $unwind$nsk_ldisplay       0000000180006330     libsetlocal004.obj
 0002:00002338       $unwind$nsk_lvdisplay      0000000180006338     libsetlocal004.obj
 0002:00002338       $unwind$_RTC_Initialize    0000000180006338     MSVCRT:initsect.obj
 0002:00002338       $unwind$_RTC_Terminate     0000000180006338     MSVCRT:initsect.obj
 0002:00002338       $unwind$?__scrt_initialize_thread_safe_statics@@YAHXZ 0000000180006338     MSVCRT:thread_safe_statics.obj
 0002:00002344       $unwind$nsk_lvcomplain     0000000180006344     libsetlocal004.obj
 0002:0000235c       $unwind$nsk_ltrace         000000018000635c     libsetlocal004.obj
 0002:0000235c       $unwind$__report_gsfailure 000000018000635c     MSVCRT:gs_report.obj
 0002:00002364       $unwind$Agent_Initialize   0000000180006364     libsetlocal004.obj
 0002:00002364       $unwind$Java_nsk_jvmti_SetLocalVariable_setlocal004_getReady 0000000180006364     libsetlocal004.obj
 0002:00002364       $unwind$nsk_lvtrace        0000000180006364     libsetlocal004.obj
 0002:00002364       $unwind$__raise_securityfailure 0000000180006364     MSVCRT:gs_report.obj
 0002:00002364       $unwind$__scrt_initialize_crt 0000000180006364     MSVCRT:utility.obj
 0002:00002364       $unwind$__scrt_initialize_onexit_tables 0000000180006364     MSVCRT:utility.obj
 0002:00002364       $unwind$__scrt_release_startup_lock 0000000180006364     MSVCRT:utility.obj
 0002:00002364       $unwind$__scrt_uninitialize_crt 0000000180006364     MSVCRT:utility.obj
 0002:00002364       $unwind$_onexit            0000000180006364     MSVCRT:utility.obj
 0002:0000236c       $unwind$nsk_lverify        000000018000636c     libsetlocal004.obj
 0002:0000237c       $unwind$nsk_vprintf        000000018000637c     libsetlocal004.obj
 0002:0000238c       $unwind$nsk_printf         000000018000638c     libsetlocal004.obj
 0002:00002394       $unwind$?nsk_jni_lverify@@YAHHPEAUJNIEnv_@@HQEBDH1ZZ 0000000180006394     libsetlocal004.obj
 0002:000023a8       $unwind$?nsk_jni_check_exception@@YAHPEAUJNIEnv_@@QEBDH@Z 00000001800063a8     libsetlocal004.obj
 0002:000023c4       $unwind$Java_nsk_jvmti_unit_FollowReferences_FollowRefObjects_resetTags 00000001800063c4     libsetlocal004.obj
 0002:000023c4       $unwind$addRefToVerify     00000001800063c4     libsetlocal004.obj
 0002:000023c4       $unwind$nsk_jvmti_resetAgentData 00000001800063c4     libsetlocal004.obj
 0002:000023c4       $unwind$nsk_jvmti_setFailStatus 00000001800063c4     libsetlocal004.obj
 0002:000023c4       $unwind$__scrt_initialize_default_local_stdio_options 00000001800063c4     MSVCRT:default_local_stdio_options.obj
 0002:000023c4       $unwind$?dllmain_crt_dispatch@@YAHQEAUHINSTANCE__@@KQEAX@Z 00000001800063c4     MSVCRT:dll_dllmain.obj
 0002:000023c4       $unwind$DllMain            00000001800063c4     MSVCRT:dll_dllmain_stub.obj
 0002:000023c4       $unwind$__GSHandlerCheck   00000001800063c4     MSVCRT:gshandler.obj
 0002:000023c4       $unwind$?__scrt_uninitialize_thread_safe_statics@@YAXXZ 00000001800063c4     MSVCRT:thread_safe_statics.obj
 0002:000023c4       $unwind$__scrt_acquire_startup_lock 00000001800063c4     MSVCRT:utility.obj
 0002:000023c4       $unwind$__scrt_dllmain_after_initialize_c 00000001800063c4     MSVCRT:utility.obj
 0002:000023c4       $unwind$__scrt_dllmain_before_initialize_c 00000001800063c4     MSVCRT:utility.obj
 0002:000023c4       $unwind$__scrt_dllmain_crt_thread_attach 00000001800063c4     MSVCRT:utility.obj
 0002:000023c4       $unwind$__scrt_dllmain_crt_thread_detach 00000001800063c4     MSVCRT:utility.obj
 0002:000023c4       $unwind$__scrt_dllmain_uninitialize_c 00000001800063c4     MSVCRT:utility.obj
 0002:000023c4       $unwind$__scrt_dllmain_uninitialize_critical 00000001800063c4     MSVCRT:utility.obj
 0002:000023c4       $unwind$atexit             00000001800063c4     MSVCRT:utility.obj
 0002:000023cc       $unwind$nsk_jvmti_lverify  00000001800063cc     libsetlocal004.obj
 0002:000023e0       $unwind$exitOnError        00000001800063e0     libsetlocal004.obj
 0002:000023f0       $unwind$Java_nsk_share_jvmti_ArgumentHandler_getAgentOptionsString 00000001800063f0     libsetlocal004.obj
 0002:00002404       $unwind$Java_nsk_jvmti_unit_FollowReferences_FollowRefObjects_getTag 0000000180006404     libsetlocal004.obj
 0002:00002404       $unwind$Java_nsk_share_jvmti_DebugeeClass_checkStatus 0000000180006404     libsetlocal004.obj
 0002:00002404       $unwind$agentThreadWrapper 0000000180006404     libsetlocal004.obj
 0002:00002414       $unwind$startAgentThreadWrapper 0000000180006414     libsetlocal004.obj
 0002:00002430       $unwind$syncDebuggeeStatus 0000000180006430     libsetlocal004.obj
 0002:00002430       $unwind$__scrt_dllmain_exception_filter 0000000180006430     MSVCRT:utility.obj
 0002:00002444       $unwind$Java_nsk_share_jvmti_DebugeeClass_resetAgentData 0000000180006444     libsetlocal004.obj
 0002:0000244c       $unwind$MA_checkStatus     000000018000644c     libsetlocal004.obj
 0002:00002460       $unwind$Java_nsk_jvmti_unit_FollowReferences_FollowRefObjects_setTag 0000000180006460     libsetlocal004.obj
 0002:00002478       $unwind$Java_nsk_jvmti_unit_FollowReferences_FollowRefObjects_addRefToVerify 0000000180006478     libsetlocal004.obj
 0002:00002494       $unwind$check_error        0000000180006494     libsetlocal004.obj
 0002:0000249c       $unwind$Breakpoint         000000018000649c     libsetlocal004.obj
 0002:000024bc       $unwind$capture_previous_context 00000001800064bc     MSVCRT:gs_report.obj
 0002:000024c8       $unwind$__GSHandlerCheckCommon 00000001800064c8     MSVCRT:gshandler.obj
 0002:000024d0       $xdatasym                  00000001800064d0     MSVCRT:amdsecgs.obj
 0002:000024d4       $unwind$?dllmain_crt_process_attach@@YAHQEAUHINSTANCE__@@QEAX@Z 00000001800064d4     MSVCRT:dll_dllmain.obj
 0002:00002510       $unwind$?fin$0@?0??dllmain_crt_process_attach@@YAHQEAUHINSTANCE__@@QEAX@Z@4HA 0000000180006510     MSVCRT:dll_dllmain.obj
 0002:00002510       $unwind$?fin$0@?0??dllmain_crt_process_detach@@YAH_N@Z@4HA 0000000180006510     MSVCRT:dll_dllmain.obj
 0002:00002510       $unwind$?fin$1@?0??dllmain_crt_process_detach@@YAH_N@Z@4HA 0000000180006510     MSVCRT:dll_dllmain.obj
 0002:00002518       $unwind$?dllmain_crt_process_detach@@YAH_N@Z 0000000180006518     MSVCRT:dll_dllmain.obj
 0002:0000256c       $unwind$?dllmain_dispatch@@YAHQEAUHINSTANCE__@@KQEAX@Z 000000018000656c     MSVCRT:dll_dllmain.obj
 0002:00002594       $unwind$?filt$0@?0??dllmain_dispatch@@YAHQEAUHINSTANCE__@@KQEAX@Z@4HA 0000000180006594     MSVCRT:dll_dllmain.obj
 0002:0000259c       $unwind$_DllMainCRTStartup 000000018000659c     MSVCRT:dll_dllmain.obj
 0002:000025ac       $unwind$__scrt_is_nonwritable_in_current_image 00000001800065ac     MSVCRT:utility.obj
 0002:000025cc       $unwind$__scrt_is_nonwritable_in_current_image$filt$0 00000001800065cc     MSVCRT:utility.obj
 0002:000025d4       $unwind$__scrt_fastfail    00000001800065d4     MSVCRT:utility_desktop.obj
 0002:000025e4       $unwind$__security_init_cookie 00000001800065e4     MSVCRT:gs_support.obj
 0002:000025f0       $unwind$__isa_available_init 00000001800065f0     MSVCRT:cpu_disp.obj
 0002:00002600       $xdatasym                  0000000180006600     MSVCRT:guard_dispatch.obj
 0002:00002608       $xdatasym                  0000000180006608     MSVCRT:guard_xfg_dispatch.obj
 0002:00002610       .edata                     0000000180006610     setlocal004.exp
 0002:00002638       rgpv                       0000000180006638     setlocal004.exp
 0002:00002678       rgszName                   0000000180006678     setlocal004.exp
 0002:000026b8       rgwOrd                     00000001800066b8     setlocal004.exp
 0002:000026d8       szName                     00000001800066d8     setlocal004.exp
 0002:000026e8       $N00001                    00000001800066e8     setlocal004.exp
 0002:000026f7       $N00002                    00000001800066f7     setlocal004.exp
 0002:00002704       $N00003                    0000000180006704     setlocal004.exp
 0002:00002739       $N00004                    0000000180006739     setlocal004.exp
 0002:0000276c       $N00005                    000000018000676c     setlocal004.exp
 0002:000027b1       $N00006                    00000001800067b1     setlocal004.exp
 0002:000027ee       $N00007                    00000001800067ee     setlocal004.exp
 0002:00002836       $N00008                    0000000180006836     setlocal004.exp
 0002:00002876       $N00009                    0000000180006876     setlocal004.exp
 0002:000028b3       $N00010                    00000001800068b3     setlocal004.exp
 0002:000028ee       $N00011                    00000001800068ee     setlocal004.exp
 0002:0000291c       $N00012                    000000018000691c     setlocal004.exp
 0002:0000294d       $N00013                    000000018000694d     setlocal004.exp
 0002:0000297c       $N00014                    000000018000697c     setlocal004.exp
 0002:000029ab       $N00015                    00000001800069ab     setlocal004.exp
 0002:000029e0       $N00016                    00000001800069e0     setlocal004.exp
 0002:00002dea       .idata$6                   0000000180006dea     kernel32:KERNEL32.dll
 0002:00002e4e       .idata$6                   0000000180006e4e     vcruntime:VCRUNTIME140.dll
 0002:00002fba       .idata$6                   0000000180006fba     ucrt:api-ms-win-crt-runtime-l1-1-0.dll
 0002:00002fdc       .idata$6                   0000000180006fdc     ucrt:api-ms-win-crt-stdio-l1-1-0.dll
 0002:00002ffc       .idata$6                   0000000180006ffc     ucrt:api-ms-win-crt-string-l1-1-0.dll
 0003:00000000       ?codeAttributeName@@3PEBDEB 0000000180008000     libsetlocal004.obj
 0003:00000008       ?lineNumberAttributeName@@3PEBDEB 0000000180008008     libsetlocal004.obj
 0003:00000010       ?localVarAttributeName@@3PEBDEB 0000000180008010     libsetlocal004.obj
 0003:00000018       ?localVarTypeAttributeName@@3PEBDEB 0000000180008018     libsetlocal004.obj
 0003:00000020       ?stackMapAttributeName@@3PEBDEB 0000000180008020     libsetlocal004.obj
 0003:00000028       ?callBytes@@3PAEA          0000000180008028     libsetlocal004.obj
 0003:0000002c       ?allocBytes@@3PAEA         000000018000802c     libsetlocal004.obj
 0003:0001aad4       redefineAttempted          0000000180022ad4     libsetlocal004.obj
 0003:0001aad8       nsk_context                0000000180022ad8     libsetlocal004.obj
 0003:0001aae4       redefineSucceed            0000000180022ae4     libsetlocal004.obj
 0003:0001aae8       agentFailed                0000000180022ae8     libsetlocal004.obj
 0003:0001aaec       currentAgentStatus         0000000180022aec     libsetlocal004.obj
 0003:0001aaf0       context                    0000000180022af0     libsetlocal004.obj
 0003:0001aba8       agentThread                0000000180022ba8     libsetlocal004.obj
 0003:0001abb0       agentThreadProc            0000000180022bb0     libsetlocal004.obj
 0003:0001abb8       agentThreadArg             0000000180022bb8     libsetlocal004.obj
 0003:0001abc0       agent_data                 0000000180022bc0     libsetlocal004.obj
 0003:0001abd0       jvmti_env                  0000000180022bd0     libsetlocal004.obj
 0003:0001abd8       jvm                        0000000180022bd8     libsetlocal004.obj
 0003:0001abe0       jni_env                    0000000180022be0     libsetlocal004.obj
 0003:0001abe8       checkStatus_func           0000000180022be8     libsetlocal004.obj
 0003:0001abf0       ?codeAttributeIndex@@3GA   0000000180022bf0     libsetlocal004.obj
 0003:0001abf2       printdump                  0000000180022bf2     libsetlocal004.obj
 0003:0001abf4       ?lineNumberAttributeIndex@@3GA 0000000180022bf4     libsetlocal004.obj
 0003:0001abf8       ?localVarAttributeIndex@@3GA 0000000180022bf8     libsetlocal004.obj
 0003:0001abfc       ?localVarTypeAttributeIndex@@3GA 0000000180022bfc     libsetlocal004.obj
 0003:0001ac00       ?stackMapAttributeIndex@@3GA 0000000180022c00     libsetlocal004.obj
 0003:0001ac04       ?stackFrameOffset@@3GA     0000000180022c04     libsetlocal004.obj
 0003:0001ac08       ?mode@@3HA                 0000000180022c08     libsetlocal004.obj
 0003:0001ac0c       ?constantPoolSize@@3GA     0000000180022c0c     libsetlocal004.obj
 0003:0001ac10       ?orig@@3PEBEEB             0000000180022c10     libsetlocal004.obj
 0003:0001ac18       ?gen@@3PEAEEA              0000000180022c18     libsetlocal004.obj
 0003:0001ac20       ?inputPos@@3PEAEEA         0000000180022c20     libsetlocal004.obj
 0003:0001ac28       ?endPos@@3PEBEEB           0000000180022c28     libsetlocal004.obj
 0003:0001ac30       ?genPos@@3PEAEEA           0000000180022c30     libsetlocal004.obj
 0003:0001ac38       ?markPos@@3PEAEEA          0000000180022c38     libsetlocal004.obj
 0003:0001ac40       ?constantPool@@3PEAPEADEA  0000000180022c40     libsetlocal004.obj
 0003:0001ac48       ?constantPoolCount@@3GA    0000000180022c48     libsetlocal004.obj
 0003:0001ac4c       ?zeroBytes@@3PAEA          0000000180022c4c     libsetlocal004.obj
 0003:0001ac50       ?codeLength@@3IA           0000000180022c50     libsetlocal004.obj
 0003:0001ac54       result                     0000000180022c54     libsetlocal004.obj
 0003:0001ac58       ?map@@3PEAIEA              0000000180022c58     libsetlocal004.obj
 0003:0001ac60       ?widening@@3PEACEA         0000000180022c60     libsetlocal004.obj
 0003:0001ac68       jvmti                      0000000180022c68     libsetlocal004.obj
 0003:0001ac70       caps                       0000000180022c70     libsetlocal004.obj
 0003:0001ac80       callbacks                  0000000180022c80     libsetlocal004.obj
 0003:0001adc0       GS_ExceptionRecord         0000000180022dc0     MSVCRT:gs_report.obj
 0003:0001ae60       GS_ContextRecord           0000000180022e60     MSVCRT:gs_report.obj
 0003:0001b330       ?g_tss_cv@@3U_RTL_CONDITION_VARIABLE@@A 0000000180023330     MSVCRT:thread_safe_statics.obj
 0003:0001b338       ?g_tss_event@@3PEAXEA      0000000180023338     MSVCRT:thread_safe_statics.obj
 0003:0001b340       ?g_tss_mutex@@3U_RTL_CRITICAL_SECTION@@A 0000000180023340     MSVCRT:thread_safe_statics.obj
 0003:0001b368       ?g_sleep_condition_variable_cs@@3P6AHPEAU_RTL_CONDITION_VARIABLE@@PEAU_RTL_CRITICAL_SECTION@@K@ZEA 0000000180023368     MSVCRT:thread_safe_statics.obj
 0003:0001b370       ?g_wake_all_condition_variable@@3P6AXPEAU_RTL_CONDITION_VARIABLE@@@ZEA 0000000180023370     MSVCRT:thread_safe_statics.obj
 0003:0001b37c       ?__proc_attached@@3HA      000000018002337c     MSVCRT:dll_dllmain.obj
 0003:0001b390       ?is_initialized_as_dll@@3_NA 0000000180023390     MSVCRT:utility.obj
 0003:0001b391       ?module_local_atexit_table_initialized@@3_NA 0000000180023391     MSVCRT:utility.obj
 0003:0001b398       ?module_local_atexit_table@@3U_onexit_table_t@@A 0000000180023398     MSVCRT:utility.obj
 0003:0001b3b0       ?module_local_at_quick_exit_table@@3U_onexit_table_t@@A 00000001800233b0     MSVCRT:utility.obj
